:1000000000610000000A0000AABE0000000000001D
:1000100000000000000000000000000000000000E0
:1000200078FFE4B8200118F6D8F99000007F007E30
:1000300007E4F0A3DFFCDEFA75817A022381121A4D
:10004000861220529002117401F022022C5774AAD9
:100050007583F5758255A574557583FA7582AAA5C1
:1000600074A57583F5758255A52200021E4A90403D
:100070007FE493FF64326003EF7002002253A87F95
:100080000080FD0219031210A9902EC27412F074A0
:100090000F121160E4F0A37402F022022C54E7095D
:1000A000F608DFFA8046E709F208DFFA803E888228
:1000B0008C83E709F0A3DFFA8032E309F608DFFA60
:1000C0008078E309F208DFFA807088828C83E30984
:1000D000F0A3DFFA806489828A83E0A3F608DFFA5E
:1000E000805889828A83E0A3F208DFFA804C80D2AC
:1000F00080FA80C680D4806980F28033801080A628
:1001000080EA809A80A880DA80E280CA803389827F
:100110008A83ECFAE493A3C8C582C8CCC583CCF02B
:10012000A3C8C582C8CCC583CCDFE9DEE7800D89D2
:10013000828A83E493A3F608DFF9ECFAA9F0EDFBD9
:100140002289828A83ECFAE0A3C8C582C8CCC58321
:10015000CCF0A3C8C582C8CCC583CCDFEADEE8807A
:10016000DB89828A83E493A3F208DFF980CC88F0EC
:10017000EF60010E4E60C388F0ED2402B40400501D
:10018000B9F582EB2402B4040050AF232345822347
:100190009008CE73EF8DF0A4A8F0CF8CF0A428CEF9
:1001A0008DF0A42EFE22C2D5EC30E709B2D5E4C30F
:1001B0009DFDE49CFCEE30E715B2D5E4C39FFFE45F
:1001C0009EFE120BF2C3E49DFDE49CFC8003120B27
:1001D000F230D507C3E49FFFE49EFE22C5F0F8A3EA
:1001E000E028F0C5F0F8E582158270021583E0384A
:1001F000F022BB010A89828A83E0F5F0A3E0225055
:100200000687F009E71922BBFE07E3F5F009E319B9
:100210002289828A83E493F5F074019322BB01075B
:1002200089828A830209BC500B09C5F027F7C5F003
:100230001937F722BBFE0D09F8E325F0F3C5F019D5
:10024000E338F322F889828A8374019325F0C5F09C
:10025000F8E4933822BB010A89828A83F0E5F0A38F
:10026000F0225006F709A7F01922BBFE06F3E5F0CD
:1002700009F3192275F008758200EF2FFFEE33FEA7
:10028000CD33CDCC33CCC58233C5829BED9AEC996E
:10029000E58298400CF582EE9BFEED9AFDEC99FC10
:1002A0000FD5F0D6E4CEFBE4CDFAE4CCF9A8822257
:1002B000B800C1B90059BA002DEC8BF084CFCECD77
:1002C000FCE5F0CBF97818EF2FFFEE33FEED33FDB0
:1002D000EC33FCEB33FB10D703994004EB99FB0F95
:1002E000D8E5E4F9FA227818EF2FFFEE33FEED336C
:1002F000FDEC33FCC933C910D7059BE99A4007ECE4
:100300009BFCE99AF90FD8E0E4C9FAE4CCFB22752A
:10031000F010EF2FFFEE33FEED33FDCC33CCC833BE
:10032000C810D7079BEC9AE899400AED9BFDEC9A20
:10033000FCE899F80FD5F0DAE4CDFBE4CCFAE4C898
:10034000F922EB9FF5F0EA9E42F0E99D42F0EC6461
:1003500080C864809845F022EB9FF5F0EA9E42F059
:10036000E99D42F0E89C45F022E8600FECC313FCE5
:10037000ED13FDEE13FEEF13FFD8F122ECF0A3ED29
:10038000F0A3EEF0A3EFF022A8828583F0D083D013
:1003900082120B7F120B7F120B7F120B7FE473E430
:1003A00093A3C583C5F0C583C8C582C8F0A3C58320
:1003B000C5F0C583C8C582C822EC8EF0A4CCC5F0B8
:1003C000CCCDF8EFA4CEC5F02DFDE43CFCE8A42E86
:1003D000C8C5F03DFDE43CFCEFA4FFE5F028FEE4D9
:1003E0003DFDE43CFC22EF4E6012EF60010EEDBBE0
:1003F000010B89828A83F0A3DFFCDEFA2289F050A8
:1004000007F709DFFCA9F022BBFEFCF309DFFCA91A
:10041000F022BC000BBE0029EF8DF084FFADF0226E
:10042000E4CCF875F008EF2FFFEE33FEEC33FCEE72
:100430009DEC984005FCEE9DFE0FD5F0E9E4CEFD65
:1004400022EDF8F5F0EE8420D21CFEADF075F00838
:10045000EF2FFFED33FD4007985006D5F0F222C391
:1004600098FD0FD5F0EA22208A03020FCF900214E4
:10047000E07002A3E06003020FCF900171E0700210
:10048000A3E06003020FCF12114A6003020FCF9066
:100490000132E0703090011D120FE4FFAEF09001C8
:1004A0000B120FE4D39FE5F09E4003020FCF121012
:1004B0004AE490017DF0A3F01211AD9002181211E0
:1004C000C4F5758003757500757614E4F5B2F5BA58
:1004D000900181E0F55DA3E0F55EC209758D2043D2
:1004E0008D20758D8043AA08D2AF758B02758EAFB3
:1004F00020062412114A701F200C1CE5DB20E21795
:10050000758AC4200C0DE5DB20E208758703000026
:10051000008006D2098002D209758B11758A50536A
:10052000AAF7D3900213E09490900212E094014055
:100530000EA3E02470F0900212E034FEF08007E495
:10054000900212F0A3F0D390021FE0949090021E4C
:10055000E09401400EA3E02470F090021EE034FE0F
:10056000F08007E490021EF0A3F01229BD90005520
:10057000E075F006A4902EC3F0A3E4F0A3F01210EF
:100580002153997F1208661210B3902EC0E030E21A
:10059000F9902EC0E4F0902E02E0F577A3E0F57814
:1005A0004389021210274380021210B0902EC0E03F
:1005B00030E2F91211D8F522A3E0F523E5782527DA
:1005C000FFE5773526FEC3EF9523F525EE9522F559
:1005D0002412118AE5259FE5249E40048E248F2550
:1005E000902EC4E4F043998090016FE524F0A3E5D8
:1005F00025F0C3E55E9525FFE55D9524FE122C35BB
:100600008E5F8F601211EB4003020FA8AE24AF255E
:100610007C007D14120B991211F5AF74AE73AD729C
:10062000AC719002C4121007FBD3120B389002C4B5
:1006300040171210FC9574FFEE9573FEED9572FD58
:10064000EC9571FC1211F58007120B680000000098
:10065000E47F607EEAFDFC9002C4121007FBD31217
:100660000B38400A9002C4120B680000EA60120FB7
:10067000E1FFAEF07C007D09120B999002C41210CC
:10068000072FFFEA3EFEE93DFDE83CFC12116E1229
:1006900011F5900132E07033AE5DAF5EFC7D091262
:1006A0001129E4FCFDEB2525FFEA35241210771211
:1006B000116E8E5D8F5E9002C4120FF21210361210
:1006C00010E3120FFC121036020FA81210E3120FE3
:1006D000FC12103690010E120FE4FFAEF09002C42F
:1006E000121004FBD3120B385003020FB8120FD0B4
:1006F000121143FEC3EF957AEE95795003020FB8BD
:1007000090010B120FE4FFAEF07C007D02120B99FA
:10071000C8ECC8EDC0E0EEC0E0EFC0E0120FD012B0
:100720001143FEE4FCFDD0E0FBD0E0FAD0E0F9EBB1
:100730002FFFEA3E1210777B0312117090010B120B
:100740000FFC1210A290010B120FE4D39430E5F0CD
:1007500094754008747575F030120A35900184E084
:100760006066121151406190010B120FE4121143A7
:10077000FE122C359002C8EEF0A3EFF090010B12A0
:100780000FE4FFC312103E50199002C9E0941E906E
:1007900002C8E09400400B120FF9F9E475F005125D
:1007A00009FD900185E0602090010B120FE412100A
:1007B0003C4015D39002C9E094289002C8E0940010
:1007C0004006120FF91211E220090D1211EB500828
:1007D00012114A7003020CBC900183E00412111143
:1007E0001210129001337401F09002161211772248
:1007F00090010EE0FBA3E0FAA3E0F91209D2FFAEEC
:10080000F0900108E0FBA3E0FAA3E0F90209D2901E
:100810000134A3A3E0F9A3E0FF90010EE0FBA3E005
:10082000FAA3E022E4FCFDE0F8A3E0F9A3E0FAA3D8
:10083000E0227A0079667E007F0B7D007B00020B50
:10084000C643AB025389FD5395FD5396FD22A3F099
:10085000A37401F0A322C98FF0020A35D3FF9001DF
:1008600089E09F900188E095F0227F087A01793431
:100870007E007D007B01020BC6E50A25E02428F8F6
:10088000E6FE08E622A3F0A37403F0A374E8F022C6
:10089000F9EB2FFFEA35F0FEED39FDEC38FC22A331
:1008A000E0FEA3E0FBCAEECAE4F9F822902E427DF6
:1008B00014E0FEA3E0FF7C00020974F9E4F5F00205
:1008C0000A35F9EE8FF0020A35902EC07402F0223C
:1008D000122C20902EC07419F022E50D25E024750D
:1008E000F582E43401F583E0FEA3E0FF229002C626
:1008F000E0FEA3E0FF2290018AE0FCA3E0FDC3EF4D
:100900009DFF229002C4A3A3E0F9A3E0FF90010899
:10091000229002147402F0A37458F022E0FCA3E0C9
:10092000FDA3E0FEA3E022900186F0A3F0A3F0A3D4
:1009300022F07E007F057D007B007A007961020B4A
:10094000C6FFE5F0F0A3EFF022120B99C8ECC8C97E
:10095000EDC9CAEECACBEFCB22E4F50EF50DF50CCE
:10096000F50B22C39FFFE5F09E2290001BE0642060
:1009700022900188E0FEA3E0FFD39400EE940022D1
:10098000902ECAF0902EC77401F0902EC4227B0ADC
:10099000E4FAF9F8020A90E4F0A374C8F022AB0E6E
:1009A000AA0DA90CA80BD3020B38E5272488FFE574
:1009B000263413FED32290016FE56CF0A3E56DF0B1
:1009C0002225E02428F8A60F08A61022E490021A97
:1009D000F0A3F022F9746175F0A8020A3590003A8C
:1009E0007410F022F0A3F0900220F0A3F022FEEFAA
:1009F0002401FFE43EC31322902EC0E4F0902E1E8B
:100A0000E022F974FF75F0FB0209FDC3E5609576FD
:100A1000E55F9575229002C4020B5C90018C121068
:100A200007FBE9C0E0EAC0E0EBC0E0900123120F51
:100A3000E4FFE4FCFDD0E0FBD0E0FAD0E01210705F
:100A400090018C120B5C900191E004F07006900113
:100A500090E004F0900192E07002A3E060030213C2
:100A6000C390018C1210FCFFEEC0E0EFC0E012104A
:100A70007FD0E0FFD0E0FE120A9090018C120B5C58
:100A800090018CA3A3E0FFA3E090018ACFF0A3EF35
:100A9000F0A3120B6800000000E490019012110A0C
:100AA00074C8F0900212E07002A3E060030213C366
:100AB000900132E07003021355900186E0FEA3E03E
:100AC000FF4E702290018AE0FDA3E0900186CDF0F8
:100AD000A3EDF090010B120FE4FD900188E5F0F01A
:100AE000A3EDF002133E1210D6EE9CFE122C3590B0
:100AF0000198120FFC1210A2900184E07026900160
:100B000098120FE4C39412E5F09400500F90010B7B
:100B1000120FE4FF9001881211228020900184744A
:100B200001F08018900198120FE4C39402E5F0944C
:100B3000005009E4121107F0900184F090018AE05E
:100B4000FEA3E0FFD3900187E09F900186E09E40E6
:100B500007E4900185F080069001857401F0E4902F
:100B60000194F0A3F090019EF090019B120FFC12F3
:100B7000109B0213C3900194E0FEA3E0FF4E70129D
:100B800090018AE0FDA3E0900194CDF0ED12106594
:100B900080511210D6EE9CFE122C3590019B120F44
:100BA000FC1210A2900196E07002A3E07035900153
:100BB0009B120FE4D39419E5F09400400C90019639
:100BC0007413F0A37488F0800BE490019EF0900100
:100BD0009612106890018AE0FFA3E0900194CFF094
:100BE000A3EFF0900132E07008121107F090018439
:100BF000F0221210A9902EC4E4F0A3F053997FF5CF
:100C00000BF50CF50DF50EF50A12086612102112FF
:100C100010B3902EC0E030E2F9902EC0E4F043898A
:100C200002121027438002902E02E0FEA3E0250C62
:100C3000F50CEE350BF50B1210B0902EC0E030E243
:100C4000F91211D8FEA3E0250EF50EEE350DF50DC7
:100C5000050AE50AC3940640B0439980902EC5E486
:100C6000F0E527240CFFE52634FEFED3EF950CEECD
:100C7000950B4015900171E07002A3E07012900195
:100C80007104F0A374F4F08007E4900171F0A3F014
:100C9000E50C2527FFE50B3526FEC3EF950EF51075
:100CA000EE950DF50F12118AE5109FE50F9E400499
:100CB0008E0F8F10900167E50FF0A3E510F0900103
:100CC0006BE50DF0A3E50EF0A3E50BF0A3E50CF04A
:100CD000AF10AE0F12229090016FEEF0A3EFF090E4
:100CE000001BE0B4200312101290016FE0FEA3E09D
:100CF000FFE4FCFDE5692FF569E5683EF568ED3533
:100D000067F567EC3566F566056BE56B7002056A9D
:100D1000C3E56F94E8E56E9403402AAE6AAF6BCBEF
:100D2000EFCB121085AF69AE68AD67AC66120A9062
:100D30008E6C8F6DE4F569F568F567F566F56AF513
:100D40006BF56EF56FD3E56D9400E56C940040593A
:100D5000900170E0956DFF90016FE0956CFE900240
:100D6000CAF0A3EFF0D394F9EE6480947F4015E0CD
:100D700094079002CAE0648094805008121196E4AF
:100D8000F57080259002CAE0FEA3E0FF122C35D357
:100D9000EF9414EE648094804003757003E570C393
:100DA00094035005121196057090016FE0F550A361
:100DB000E0F55178287C007D007B007A00792A7E5E
:100DC000007F2802094E120FD0FDACF0D39FEC9E9D
:100DD000403490010E120FE4FFC3ED9FFFEC95F03D
:100DE000FED3EF9430EE9475400D9002C67475F00A
:100DF000A37430F0021629120FDB1211439002C6C1
:100E0000F0A3EFF08043120FE1FFAEF090010E125D
:100E10000FE4FDACF0C39FFFEC9EFED3EF9410EE09
:100E20009427400C9002C674D8F0A374F0F080129E
:100E3000120FE1FFC3ED9FFEEC95F09002C6F0A308
:100E4000CEF0E49002C6F0A3F0900132E0605012C0
:100E500010CDD39400EE64809480401A900120124B
:100E60000FE4FDD3EF9DEE95F0400B900218E4F0F7
:100E7000A37464F0801BD3900219E09400900218D0
:100E8000E09400400C90010B120FE49002C6121186
:100E900021D20B90021E740FF0A374A0F0800D906D
:100EA000021C1210687A007952121016D39002C7F1
:100EB000E094009002C6E0648094805003021750D2
:100EC000E0F9A3E0FF90010B120FFC121036121094
:100ED000CDEE3395E0FDFCE47BB87A88F9F8C312D7
:100EE0000B22500A9002C67488F0A374B8F0D39015
:100EF000021BE0940090021AE09400500790001B3F
:100F0000E0B4201D1210CDC39496EE6480948050FE
:100F100010EF9400EE6480948040257C007D0A8070
:100F20001430001C1210CDC394A0EE6480948F5036
:100F30000F7C007D321209869002C6EEF0A3EFF01E
:100F4000900132E0600C90021CE07002A3E070029D
:100F500080009002C6E0F9A3E0FF900114120FFC9C
:100F6000121036900114120FE424A8FFE5F0801D42
:100F700090010B120FFC12109B900114120FFC1227
:100F8000109B9002C7E024A8FF9002C6E03461F9EC
:100F9000900111120FFC12103622900132E0700302
:100FA00002181712104A900216121068900184E07D
:100FB0007003021902121151500302190290010B21
:100FC000120FE4121143FE122C359002C6EEF0A36C
:100FD000EFF0D39496EE9400400CE4900184F090EE
:100FE0000186F0A3F022900185E0602090010B12B1
:100FF0000FE412103C4015D39002C7E094289002F1
:10100000C6E094004006120FF91211E290010B1293
:101010000FE4C312103D40030219029002C7E0948E
:101020001E9002C6E094005003021902120FF9F953
:10103000E475F0050209FD900134121007FBE9C0C8
:10104000E0EAC0E0EBC0E0120FE1FFE4FCFDD0E01D
:10105000FBD0E0FAD0E0121070900134120B5C90DB
:101060000139E004F07006900138E004F0900216B7
:10107000E07002A3E060030219029001341210FC38
:10108000FFEEC0E0EFC0E012107FD0E0FFD0E0FE46
:10109000120A90900134120B5C90010E120FE4249E
:1010A0001EFFE435F0FE900134121004FBD3120B46
:1010B00038403F900212E07002A3E0703590019E2C
:1010C000E0702F200B2C90013BE004F070069001A3
:1010D0003AE004F0D390013BE0940590013AE094AB
:1010E00000401E120FEF121036E490013AF0A3F008
:1010F000800F120FEF121036E490013AF0A3F0C205
:101100000B900134120B6800000000E4900138F0ED
:10111000A3F090019EE09002166004121177221253
:10112000106822C0E0C083C082C0D0D2AF90022538
:10113000E004F0D3900213E09400900212E09400D7
:10114000400CA3E024FFF0900212E034FFF0D390B3
:101150000215E09400900214E09400400CA3E024F7
:10116000FFF0900214E034FFF0D3900217E09400F7
:10117000900216E09400400CA3E024FFF0900216C9
:10118000E034FFF0D3900219E09400900218E0944C
:1011900000400CA3E024FFF0900218E034FFF0D3ED
:1011A00090021BE0940090021AE09400400CA3E02F
:1011B00024FFF090021AE034FFF0D3900223E09471
:1011C00000900222E09400400CA3E024FFF0900283
:1011D00022E034FFF0D3900221E09400900220E05E
:1011E0009400400CA3E024FFF0900220E034FFF0D4
:1011F000D390021DE0940090021CE09400400CA3E8
:10120000E024FFF090021CE034FFF0C3E56F94E8A7
:10121000E56E94035008056FE56F7002056EC3E537
:101220005B94E8E55A94035008055BE55B700205A2
:101230005AD3900193E09400900192E09400400C06
:10124000A3E024FFF0900192E034FFF0D3900197E7
:10125000E09400900196E09400400CA3E024FFF09D
:10126000900196E034FFF0D3900172E09401900178
:1012700071E09400400CA3E024FFF0900171E03491
:10128000FFF0D390021FE0940090021EE094004013
:101290000CA3E024FFF090021EE034FFF0D0D0D089
:1012A00082D083D0E0327E007FFF7D007B017A0018
:1012B0007904120BC69002D87400F0A37404F09065
:1012C00001C57401F0A37400F0A374B8F09001CBD1
:1012D0007401F0A37400F074AC1229AA7400F0A396
:1012E0007494F09001C87401F0A37400F0A374C664
:1012F000F09001D17401F0A37400F074D21229AA05
:101300007400F0A3741F1229AB7401F0A37402F0EF
:10131000902DE0E493FF9002D8E0FCA3E0FDF5827D
:101320008C83A3EFF0900002E0FFED2404122984E7
:10133000900001E0FFED2405122984900003E0FFF6
:10134000ED2406122984902DE2E493FFED2412127D
:101350002984902DE3E493FFED2414122984900155
:10136000DA7401F0A37400F0A3743CF0E4FF75F0AC
:1013700002EFA42401F582E5F0342EF583E493FE18
:1013800074542FF582E43400F583EEF0EF25E02469
:101390002DF582E4342EF583E493FE1229B2EEF0AB
:1013A0001229B2E0FEEF25E0242CF582E4342EF57C
:1013B00083E49324C0F582E4342EF583EEF00FEF3E
:1013C000B416AB902F56E0900058F0902F56E09056
:1013D000006EF0902F56E0900059F0902F56E0905C
:1013E000006FF09000FF7401F09000FEF090003A62
:1013F0007410F090001BF0900028F0A37420F0907F
:1014000002127413F0A37488F022121139F515F545
:1014100016852811852912852813852914F50A12A5
:101420001059FFD3E5149FE5139E40078E138F14C8
:10143000850A16C3E5129FE5119E50078E118F1283
:10144000850A15050AE50AB414D5E4F50FF510F57B
:101450000AE516650A602EE515650A6028E510455F
:101460000F7010E50A25E02428F8E6F50F08E6F5E8
:101470001080121210592510FFE50F3E1211CEF503
:101480000FEF13F510050AE50AB414C5900181E5C4
:101490000FF0A3E510F0E516C394115005E5161200
:1014A00011A1E515C394115005E5151211A11211F2
:1014B00039F50A121059FFC3E5109FFFE50F9EFE94
:1014C000122C35D3EF9419EE64809480400FE4FC25
:1014D000FDE50E2510F50EE50D350F800F121059A4
:1014E000FFE4FCFDE50E2FF50EE50D3EF50DED35A7
:1014F0000CF50CEC350BF50B050AE50AC39414400A
:10150000B2AF74AE73AD72AC7112117E401AE50EBB
:101510009574F50EE50D9573F50DE50C9572F50CCA
:10152000E50B9571F50B8003121139E47F607EEABB
:10153000FDFC12117E400BE4750E60750DEAF50C92
:10154000F50BAE0DAF0E2290017DE0FEA3E0FFC3D0
:101550009404EE9400502F900106E0FCA3E0FDEF10
:1015600025E0FFEE33FE74752FF58274013EF5839E
:10157000ECF0A3EDF090017EE004F0700690017DA8
:10158000E004F0021DEC750D011210BAE50D25E026
:101590002473F582E43401F583EEF0A3EFF0050D3A
:1015A000E50DB404E4120FE1FF9001061210D9E535
:1015B000F09CFE122C35C3EF9428EE64809480508A
:1015C0003C900132E0702890010E120FE4FFC390AE
:1015D0000107E09FFF900106E095F0FE122C35C355
:1015E000EF9414EE64809480500590010E80039077
:1015F0000108120FE4FF90017BE5F0800B900106DB
:10160000E0FFA3E090017BCFF0A3EFF0E4F50CF551
:101610000BF50AF509F50DD390017EE0950D9001CB
:101620007DE09400401E1210BAE4FCFDE50C2FF59D
:101630000CE50B3EF50BED350AF50AEC3509F5091D
:10164000050D80D3AF0CAE0BAD0AAC09EEC0E0EFD8
:10165000C0E090017D121080D0E0FFD0E0FE120AC1
:10166000908F0C8E0B8D0A8C0922C0E0C083C08243
:10167000C0D0ECC0E0EDC0E0EEC0E0EFC0E0D2AF23
:10168000E5DB30E419D20CC208E5DB30E102802E44
:101690009002D7E5DFF09002DAE4F0021F48E5DBC4
:1016A00030E50FD206300805C208021F48C20C02FE
:1016B0001F48C208E5DB30E13AE5DB30E01090027C
:1016C000DBE0FF04F0122C0AE0F5DF021F48900275
:1016D000DBE0FFB40813208A10D28A9002D8E0FC25
:1016E000A3E02407122C10E4F0EF641A707AD207FA
:1016F000021F489002DAE0700EA3E5DFF09002DAF4
:101700007401F0D20880619002DBE0902A2F93FFF1
:10171000B4FF089002D7E5DFF08047EF640F70292F
:101720009002DBE0FFA3E0FCA3E0FD122C0FE054ED
:101730000FF09002DBE0FF04F0ED122C0FE0FFE56C
:10174000DF54F0FEEF4EF0801F9002DBE0FF122C22
:101750000AE5DFF0EFB4240A9002147401F0A374D8
:10176000F4F09002DBE004F075DBFFD0E0FFD0E0A6
:10177000FED0E0FDD0E0FCD0D0D082D083D0E032EB
:101780009002CAEFF09002CFE4F0A374FFF0E4A35C
:10179000F0A3F0A304F0A374FFF0902EC07402F045
:1017A000902EC37408F0E49002CBF0A3F09002CB2B
:1017B000E0FEA3E0FFC39409EE9400400302204F33
:1017C000EF9407EE940040067E007F01801990029E
:1017D000CBA3E004FFE47E01C8EFC8088006CEA2D8
:1017E000E713CE13D8F8FF9002CDEEF0A3EFF09000
:1017F0002EC07419F0902EC0E030E2F99002CAE0D9
:10180000FF75F002A42400122999E0FCA3E0FD90EA
:101810002EC07402F0D3ED94FFEC940F40179002A9
:10182000CDE0FCA3E0FD75F002EF122996EC8DF0FF
:101830001209BC80299002CAE075F002122996C0F4
:1018400083C082E0FEA3E0FF9002CDE0FCA3E0FDB8
:10185000C3EF9DFFEE9CD082D083F0A3EFF0900207
:10186000CCE004F070069002CBE004F0021F8D7F04
:1018700000227F997A0179061210509001087401B4
:10188000F0A37400F0744412102E7400F074461229
:10189000102E7400F0A3744812102F7400F0A3747B
:1018A0003212102F7400F0A3742E12102F7400F057
:1018B000A3742CF09001237401F0A37400F0A374BE
:1018C00026F09001987401F0A37400F0A3748412C0
:1018D000102F7400F0A37486F09001267401F0A319
:1018E0007400F0A3741C12102F7400F0A37422F083
:1018F00090011A7401F0A37400F0A3743612102F33
:101900007400F0A3742A12102F7400F0A37438F03E
:10191000757900757AC890011A120FFCF9E579857E
:101920007AF0120A3590011D120FFCF9E475F0648B
:10193000120A35900120120FFCF9E475F096020AA4
:10194000359002C6EEF0A3EF1211119002C6E070BE
:1019500002A3E060031221D91226B0E490017DF0C9
:10196000A3F07F14122A659002147402F0745812C6
:101970001065900106E0F9A3E0FFA3120FFC12101E
:101980003690010B120FFC12109B900111120FFCEC
:101990001211B4900114120FFC12109B9001171237
:1019A0000FFC1211B41211BDE4900132F090013419
:1019B000120B6800000000E490013812110AF09048
:1019C0000106120FF4121036E4900133F090022257
:1019D0001211C490021EF0A3F0FE7F14FD7B017A69
:1019E000017984120BC6900123120FE490018A1230
:1019F000112190019212117722122B17902E42E0A2
:101A0000FEA3E024BBFFEE34FE9002C8F0A3EFF08B
:101A100012102153997F1229BD1208661210A99045
:101A20002EC314F01210B3902EC0E030E2F9902EC5
:101A3000C0E4F0902E027D121210918E268F277D29
:101A400014120B99EF24E0F574EE34B1F573ED3414
:101A5000FFF572EC34FFF5714389021210274380C1
:101A60000243998053997F122C20902E5EE4F0A3BC
:101A700074FFF07F0F121F60902E5EE0FEA3E0D394
:101A800094F0EE94014007902E5EE4F0A3F0902EC7
:101A9000C4E4F0439980A3F0900105E0900021F0A8
:101AA00012108C900126120FFCF9EE8FF0020A350D
:101AB0009002CCEEF0A3EFF0E5644563700C900269
:101AC000CCE0F563A3E0F56480169002CDE02564D8
:101AD000FF9002CCE035631211CEF563EF13F5648D
:101AE0000565E565D3940A400D856361856462E40C
:101AF000F563F564F565D3E5629400E56194004013
:101B00005C9002CDE09562FF9002CCE09561FE1200
:101B10002C35C3EF940AEE648094805028AE61AFF8
:101B2000627C007D031211299002CCE0FEA3E0FF4D
:101B3000E4FCFDEB2FFFEA3E1210777802120B490E
:101B40009002CC80139002CDE02562FF9002CCE0A1
:101B50003561C313FEEF13FFEEF0A3EFF09002CC5C
:101B6000E0FEA3E0FF22022AC0E493A3F8E493A3DB
:101B70004003F68001F208DFF48029E493A3F854CF
:101B800007240CC8C333C4540F4420C8834004F452
:101B900056800146F6DFE4800B0102040810204065
:101BA00080902536E47E019360BCA3FF543F30E56E
:101BB00009541FFEE493A360010ECF54C025E060DA
:101BC000A840B8E493A3FAE493A3F8E493A3C8C5A8
:101BD00082C8CAC583CAF0A3C8C582C8CAC583CA99
:101BE000DFE9DEE780BE30000875791B757A588022
:101BF00006757900757AC890010B120FE4FFAEF0FC
:101C0000C3957AEE95795015900132E060209001ED
:101C100020120FE4FDC3EF9DEE95F0401190021AE3
:101C2000E07002A3E0702790013204F08020900061
:101C30001BE0B420051211AC800690021A12117735
:101C4000E4900132F0900218F0A3F01211BD90015F
:101C500032E06011900028E090003AB41004741053
:101C6000F0227420F02290022FE014601B146043D5
:101C70002402705D900239E0B4010A90022F122410
:101C8000B2D205D200C203227F021228C7EF60073A
:101C90007F02122C41C205900239E0703490022F6D
:101CA0007402F0D203C205C2007F03122C417F03ED
:101CB0000227627F031228C7EF60167F03122C41B0
:101CC000900239E090022F7003F080031224B2C218
:101CD00003227401F07F02122C417F02122762223C
:101CE000CDEFCD43AD105399EF439A10539BEF9036
:101CF0002EC07402F0147E00C8EDC8088005C333FE
:101D0000CE33CED8F9FF902EC4EEF0A3EFF0902E94
:101D1000C8EEF0A3EFF07410122B73902EC0E030D9
:101D2000E2F9902EC0E4F07402F07420122B73904C
:101D30002EC0E030E2F9902E00E0FEA3E0FF902EEE
:101D4000C4E4F0A3F0902EC0F0439910539AEF53DF
:101D50009BEF5390EF22C10C41023300410234004B
:101D60004102300041023800C102C101C1044102F8
:101D7000390041022F00C103C100C1054102DA0050
:101D80004102DB004202D50000C106C108C1074183
:101D900002D7104101030041010510C10BC10A41E6
:101DA000019F0002260000047100000000410104B0
:101DB0001041023A00009002C47408F0A3E4F0A3BA
:101DC000743FF0A374DFF0E4FDFCF9758A10538AC8
:101DD000EF009002C4E0FEA3E02DF582EE3CF58317
:101DE000E493FF69F90DBD00010CBC37E5BDDFE2EE
:101DF0009002C6122C17E493699002D87009122C35
:101E000017A3740AF08006122C17A3E4F0758A5009
:101E1000538AEF0022200A06200303300509E4FF5D
:101E2000FE122121C20A22900220E07002A3E0608B
:101E30000512114A703A2000031229F61226B07FCB
:101E400001122A65121D279002C4EEF0A3EFF07B69
:101E5000017A0279C41227FB9002C41210E8120F13
:101E6000FC1210361215A61223C61211FB12177A95
:101E700012294922900211E024FE601314602314F9
:101E80006027240370499002117402F0122C507FD5
:101E9000017E001221219002117403F0E4900230BF
:101EA000F0229002117404F0221224461227B31279
:101EB0002446900171E07004A3E06401700C90016D
:101EC00071F0A3F09002117402F0E4900225F02268
:101ED0004389025395FD5396FD438002122BAD7F3B
:101EE0000C1224C0CAEECACBEFCB7F0C1224C0EF79
:101EF0002BFFEE3A9002C9F0A3EFF0122B7FF912FC
:101F000009D245F07006122B64EE80181209D2FB3C
:101F1000AAF0122B64EF2BFFEE3AC313F9EF13FF75
:101F2000122B7FC98FF0120A35221229A2F5828E58
:101F300083A3E0B4AA031225961229A2FF12298DC9
:101F4000E0B41008EF12298DE4F0D20A1229A2FFA2
:101F5000241B12298FE0700DEF241C12298FE0B48E
:101F600010031228421229A2241312298FE0FFB471
:101F700010069002397401F0EFB42005E4900239A4
:101F8000F0229002C4EFF0E024BB122B8DE060033E
:101F90007F01229002C4E0FF24BB122B8D7401F05C
:101FA000EF122B95E493FE740193FFE4FCFD902F58
:101FB00060E0F8A3E0F9A3E0FAA3E02FFFEA3EFE19
:101FC000ED39EC389002C4E0122BA1EEF0A3EFF053
:101FD0007F002212114A702990019FE070031210B5
:101FE000F190019F7401F0900029E0B420081225BF
:101FF000F5120C478003122A939002247401F0809A
:1020000017E490019FF0900029E0B420031225F519
:10201000900224E06002E4F0022BD09002C6EBF0C4
:10202000A3EAF0A3E9F0900214E07002A3E070319B
:10203000900133E0602BE4900133F01226B01210CF
:10204000F17508017F01122A65121D279002C61240
:102050000FFC1210A20508E508C3941440E6121103
:10206000AC2212082EE4F5F275F30875EEFF75EF59
:102070003F75EA81F5F675EB0700E5EC30E7FBE428
:10208000F5EC9002D8E0FEA3E0FF241BF582E43ECD
:10209000F583E5F3F0EF241CF582E43EF583E5F2E9
:1020A000F075EB3022758B11902F647440F0E4FED4
:1020B000E4FFEF75F003A4244DF582E43402F583C8
:1020C000E5822EF582E43583F583E4F00FEFB40A60
:1020D000E10EEEB403DA7F099002BBE4F0A3DFFC6B
:1020E000902F647480F022CBEFCB122B8AE0603605
:1020F000902F60A3A3E0FEA3E0FFEB122BA1E0FC76
:10210000A3E0FDD39FEC9E501DC3EF9DFFEE9CFE10
:10211000EB122B95C37401939FE4939E4008122BFE
:102120008AE4F07F01227F0022758A50538AEF9063
:1021300000027411F09000017422F09000037433D7
:10214000F0E4F5AB75AC1DF5ADF5AF7589FF759194
:102150003F7599FFF59675931CF59BF595F592F5EE
:102160009A5388FCD28AD20D2290003AE0FC90016A
:1021700004E06C602E90003AE0FE900104F09000C4
:102180000BE0900238F0540FF0EEB42005E044204C
:10219000800AECB4100B900238E04410F090000B71
:1021A000F0C28A22F582E43CF583EFF022241AF58E
:1021B00082E43EF58322A42440F582E5F0342EF536
:1021C00083229002D8E0FEA3E022A3F0A37401F0E2
:1021D000A322746A2FF582E43400F583221210A939
:1021E000902EC4E4F0A3F0FF74542FF582E4340081
:1021F000F583E0FE75F002EFA42400F582E5F034EB
:102200002EF583E49324C0F582E4342EF583EEF0BA
:102210000FEFB416D322300735C207902E42E0FFED
:10222000A3E09002C6CFF0A3EFF0122B1712108C90
:10223000900126120FFC1210A21210A99002C6E003
:10224000FFA3E0902E42CFF0A3EFF01210F1220096
:10225000000000FFFFFFFF0000FFFFFFFFFFFFFF89
:10226000FFFF00FF000000FFFF000000FFFFFFFF77
:10227000FFFFFF00000000FFFFFFFFFFFFFFFFFF6A
:10228000FF000000009002C9EFF01229BDE4F5093B
:102290009002C9E0FFE509C39F50071213D2050958
:1022A00080EE902EC0E4F0121BEA900106EEF0A33F
:1022B000EFF022E4F5B2F5BA758D20438D20538DF1
:1022C0007F53AAF7F58BE5DB20E211200C0EE4F535
:1022D0008A758703000000758A50D20A758B112217
:1022E00012084E53A87F12290912081E122AEC4325
:1022F000A880122C4A9000FFE06006900211740141
:10230000F0122BEE12270A12265480F59002D8E024
:10231000FFA3E09002DCCFF0A3EFF0E4F5DA75DA8A
:102320004043DA2075D74075DA5875D90143A908BA
:1023300075B80875F8082212102153997F1229BD2B
:10234000902E42E4F0A374FFF01208667F01121F82
:10235000604389021210274380024399802201F4CE
:102360000028002801F4009603E801F403E8177040
:10237000006403E8003202580258012C01F403E81B
:10238000271000C89002C9E0FEA3E0FF7C007D1486
:10239000020974902EC2F0902EC0E04419F02290F1
:1023A0000123E0FBA3E0FAA3E02274BB2BF582E457
:1023B0003402F5832225E02452F582E4342BF583A0
:1023C0002225E0243BF582E43402F58322902EC0DE
:1023D0007402F0902EC77474F0902ECD74C0F0A3E8
:1023E00074FFF0A3F0902EC37401F0902ECAF02277
:1023F000E5B230E005E5AA20E013E4900226F0758E
:10240000B28E75B6F9F5B743B20143AA0122E4FFD3
:102410003006169002D8E0FCA3E0F5828C83E0FE43
:1024200054F0FFEE540FF0C20622A3E0FCA3E02F0D
:10243000F582E43CF58322E0FEA3E0F5828E832260
:102440001210A9902EC27412F074091211607480D7
:10245000F0A3E4F022EE30E707C3E49FFFE49EFE22
:102460002274BB2F122B8DE4F022122C5A022885E5
:102470001211BD22D2AF32D2AF32022BD0000000F7
:10248000000000000000000000000000000000004C
:10249000000000000000000000000000000000003C
:1024A000000000000000000000000000000000002C
:1024B000000000000000000000000000000000001C
:1024C000000000000000000000000000000000000C
:1024D00000000000000000000000000000000000FC
:1024E00000000000000000000000000000000000EC
:1024F00000000000000000000000000000000000DC
:1025000000000000000000000000000000000000CB
:1025100000000000000000000000000000000000BB
:1025200000000000000000000000000000000000AB
:10253000000000000000000000000000000000009B
:10254000000000000000000000000000000000008B
:10255000000000000000000000000000000000007B
:10256000000000000000000000000000000000006B
:10257000000000000000000000000000000000005B
:10258000000000000000000000000000000000004B
:10259000000000000000000000000000000000003B
:1025A000000000000000000000000000000000002B
:1025B000000000000000000000000000000000001B
:1025C000000000000000000000000000000000000B
:1025D00000000000000000000000000000000000FB
:1025E00000000000000000000000000000000000EB
:1025F00000000000000000000000000000000000DB
:102600000A03AB61000000000000000000000000B1
:1026100000000000000000000000000000000000BA
:10262000021203030A0F0DA00EB60FFF0C020BFFE0
:1026300023F724062504070127082A0828022B026D
:1026400029032C032D082E082F0426080211030647
:102650000A100D400E800FFF0C020BFF23F4240420
:102660002504070127102A1028042B0429032C0312
:102670002D202E202F10262000000000000000003A
:10268000000000000000000000000000000000004A
:10269000000000000000000000000000000000003A
:1026A000000000000000000000000000000000002A
:1026B000000000000000000000000000000000001A
:1037F000000000000000000000000000000000A227
:1038000000000000000000000000000000000000B8
:1038100000000000000000000000000000000000A8
:00000001FF
